:020000040800F2
:1000000000C00020911F0008011F0008031F000806
:10001000051F0008071F0008091F00080000000056
:100020000000000000000000000000000B1F00089E
:100030000D1F0008000000000F1F0008111F00081E
:10004000D91F0008D91F0008D91F0008D91F0008B0
:10005000D91F0008D91F0008D91F0008D91F0008A0
:10006000D91F0008D91F0008D91F0008D91F000890
:10007000D91F0008D91F0008D91F0008D91F000880
:10008000D91F0008D91F0008D91F0008D91F000870
:10009000D91F0008D91F0008D91F0008D91F000860
:1000A000D91F0008D91F0008D91F0008D91F000850
:1000B000D91F0008D91F0008D91F0008D91F000840
:1000C000D91F0008D91F0008D91F0008D91F000830
:1000D000D91F0008151F0008211F00082D1F000848
:1000E000D91F0008D91F0008D91F0008D91F000810
:1000F000D91F0008D91F0008D91F0008D91F000800
:10010000D91F0008D91F0008D91F0008D91F0008EF
:10011000D91F0008D91F0008391F0008D91F00087F
:10012000D91F0008D91F0008D91F0008D91F0008CF
:1001300000000000000000000000000000000000BF
:1001400000000000000000000000000000000000AF
:10015000000000000000000000000000000000009F
:10016000000000000000000000000000000000008F
:10017000000000000000000000000000000000007F
:10018000000000000000000000000000000000006F
:10019000000000000000000000000000000000005F
:1001A000000000000000000000000000000000004F
:1001B000000000000000000000000000000000003F
:1001C000000000000000000000000000000000002F
:1001D000000000000000000000000000000000001F
:0401E0005FF8E0F1F3
:1001E40010B5054C237833B9044B13B10448AFF36D
:1001F40000800123237010BD740000200000000063
:100204000431000808B5034B1BB103490348AFF39D
:10021400008008BD000000007800002004310008C0
:1002240038B50E4B054618784FF47A73B3FBF0F3E8
:100234000B4A1068B0FBF3F000F09EF8044658B97E
:100244000F2D09D8024629464FF0FF3000F054F82C
:10025400044B20461D6038BD012038BD000000203D
:100264000C00002004000020074A08B5136803208E
:1002740043F01003136000F02DF80020FFF7D0FFC7
:1002840001F076FD002008BD00200240034A044B23
:1002940011681B780B441360704700BF8401002071
:1002A40000000020014B1868704700BF8401002043
:1002B40038B50446FFF7F6FF0546631C1EBF044B22
:1002C4001B78E418FFF7EEFF401B8442FAD838BDD0
:1002D40000000020074A0002D36800F4E06023F421
:1002E400E0631B041B0C43F0BF6343F4003303437C
:1002F400D360704700ED00E0174B30B5DC68C4F301
:100304000224C4F10703251D042B28BF0423062D52
:100314004FF0010598BF002405FA03F303F1FF33FE
:1003240088BF033C1940A14005FA04F4013C224073
:10033400002842EA01024FEA0212AFBF00F1604016
:10034400064B00F00F00D2B2A5BFD2B200F5614057
:100354001A5480F8002330BD00ED00E014ED00E0F5
:100364000123420900F01F0003FA00F0014B43F897
:100374002200704700E100E00138B0F1807F0AD22A
:10038400F021064B064A586082F823100020072209
:1003940098601A6070470120704700BF10E000E0C9
:1003A40000ED00E090F8213010B5022B03D00423B7
:1003B4008363012010BD03681A6822F00E021A60DC
:1003C4001A6822F001021A60294A934224D902F5DC
:1003D4006272934219D01432934218D01432934269
:1003E40017D0143293420CBF4FF480534FF4803330
:1003F400204A53600123002480F82130436B80F8A5
:1004040020409BB39847204610BD0123F0E71023FA
:10041400EEE74FF48073EBE717498B4216D01431A3
:100424008B4215D014318B4214D014318B4214D02A
:1004340014318B4214D014318B4214D0934214BF24
:100444004FF480334FF080730C4AD2E70123FBE76B
:100454001023F9E74FF48073F6E74FF48053F3E782
:100464004FF48033F0E74FF48013EDE7184610BDE6
:1004740080000240000402400800024000000240E4
:100484002DE9F74F002216466C4F6D4BDFF8B8E1AB
:10049400DFF8B8C14FF001080C6808FA06F808EA5A
:1004A4000404A04540F085804D68122D00F0B7800B
:1004B40000F28D80022D00F0AF8000F28180002DCB
:1004C40000F09180012D00F0A5804FF00F09FF2C62
:1004D40093BF824606F18045083DD0F800B092BF34
:1004E400B500D0F804B0AD0009FA05F82BEA080805
:1004F40002FA05F588BF00F1040A48EA0505CAF8BE
:100504000050D1F804A01AF0805F52D0BD6926F0E3
:10051400030845F00105BD61BD6908F1804805F097
:100524000105019508F5803806F0030B019D4FEA9B
:100534008B0BD8F8085009FA0BF925EA0909414D43
:10054400A84271D005F58065A8426FD005F5806595
:10055400A8426DD005F58065A8426BD005F580658D
:10056400A84269D070450CBF0525062505FA0BF590
:1005740045EA0905C8F808501D681AF4803F14BFFD
:100584002543A5431D605D681AF4003F14BF25434D
:10059400A5435D609D681AF4801F14BF2543A543DD
:1005A4009D60DD681AF4001F14BF2C4325EA04047F
:1005B400DC600136102E7FF46DAF03B0BDE8F08F20
:1005C400032D25D0112D80D1CA6804327DE76545FD
:1005D40009D012D8DFF878904D4504D009F5803958
:1005E4004D457FF472AF8A68E2B1012A0CBFC0F8AE
:1005F4001080C0F81480082267E7DFF858904D4552
:10060400F1D009F580394D45EDD0A9F58019E7E71A
:1006140000225AE7CA6858E7CA68083255E7CA6828
:100624000C3252E7042250E700259FE701259DE79D
:1006340002259BE7032599E7042597E7001002406C
:100644000004014000080140001C0140000021108A
:1006540000001110000031100AB101617047090453
:10066400FBE7C3685940C1607047000003682DE987
:10067400F341DB07054610D42B689F075ED42B6833
:10068400190700F195802B685A0700F1BF80EA69C9
:10069400002A40F02D81002014E0904C636803F0A0
:1006A4000C03042B07D0636803F00C03082B0CD154
:1006B4006368DE0309D523689C03DDD56B68002BD2
:1006C400DAD1012002B0BDE8F0816B68B3F5803F58
:1006D40010D1236843F480332360FFF7E3FD06461B
:1006E40023689803C8D4FFF7DDFD801B6428F7D97D
:1006F4000320E7E79BB9236823F48033236023684E
:1007040023F480232360FFF7CDFD06462368990375
:10071400B2D5FFF7C7FD801B6428F7D9E8E7B3F526
:10072400A02F236803D143F480232360D1E723F46B
:1007340080332360236823F48023CDE7674C636808
:1007440013F00C0F07D0636803F00C03082B10D1CF
:100754006368DA030DD423689B0702D52B69012B48
:10076400AFD123686A6923F0F80343EAC203236024
:1007740085E72A695A4B6AB101221A60FFF792FD94
:10078400064623689F07ECD4FFF78CFD801B0228E4
:10079400F7D9ADE71A60FFF785FD06462368980789
:1007A4007FF56DAFFFF77EFD801B0228F6D99FE72A
:1007B400AA694A4C4B4BDAB101221A60FFF772FD69
:1007C4000646636A9B070DD54FF4FA52464B1B68E5
:1007D400B3FBF2F3019300BF019B5A1E0192002B5D
:1007E400F9D150E7FFF75EFD801B0228E9D97FE7C6
:1007F4001A60FFF757FD0646636A9F077FF543AF0C
:10080400FFF750FD801B0228F6D971E7334CE369EA
:10081400D80024D40127E36943F08053E361E369FA
:1008240003F080530093009B304E3368D90518D5EC
:10083400EB68012B26D1236A43F001032362FFF7FF
:1008440031FD41F288368046236A9B073FD5002F4D
:100854003FF41DAFE36923F08053E36117E70027FA
:10086400E2E7336843F480733360FFF71BFD80468F
:100874003368DA05DCD4FFF715FDA0EB0800642823
:10088400F6D935E7ABB9236A41F2883823F001037E
:100894002362236A23F004032362FFF703FD064661
:1008A400236A9807D3D5FFF7FDFC801B4045F7D991
:1008B4001EE7052B236A03D143F004032362BAE73E
:1008C40023F001032362236A23F00403B6E7FFF74E
:1008D400E9FCA0EB0800B042B6D909E700100240D9
:1008E40000004242800442420C000020007000409C
:1008F400224C636803F00C03082B3FF4E2AE0023A0
:100904001F4E022A33602BD1FFF7CCFC0746236825
:1009140099011FD42B6AB3F5803F05D16268A96899
:1009240022F400320A436260696A62680B4322F46B
:1009340074121343636001233360FFF7B3FC05466D
:1009440023689A013FF5A7AEFFF7ACFC401B0228D1
:10095400F6D9CDE6FFF7A6FCC01B0228D7D9C7E617
:10096400FFF7A0FC054623689B017FF594AEFFF7D3
:1009740099FC401B0228F6D9BAE600BF00100240D9
:100984006000424230B5194B87B002AC03F1100548
:10099400224618685968083303C2AB421446F7D19B
:1009A40001238DF80430022311498DF805304B687A
:1009B40003F00C02082A17D1C3F3834206A80244A9
:1009C400DB0312F8102C0CD54B680A48C3F34043E0
:1009D400504306AA134413F8143CB0FBF3F007B0D9
:1009E40030BD05485043FAE70248F8E71C310008D7
:1009F4000010024000127A0000093D00544A2DE91B
:100A0400F0411368054603F007038B420E462AD3D0
:100A140029688C0734D4CA0747D44D4A136803F0B5
:100A240007039E42C0F082802A684A4C12F0040FE9
:100A340040F08780130706D563682A6923F460535E
:100A440043EAC2036360FFF79DFF6368424AC3F34E
:100A54000313D35CD840414B18600020FFF7E0FB40
:100A64000020BDE8F081136823F007030B431360F3
:100A7400136803F007039942CAD00120BDE8F0814E
:100A8400344B11F0040F1EBF5A6842F4E0625A60FE
:100A9400080742BF5A6842F460525A605A68A8680C
:100AA40022F0F00202435A60B5E76A68294C012A31
:100AB40023681CD113F4003FDFD0636841F2883807
:100AC40023F0030313436360FFF7ECFB6B680746F3
:100AD400012B14D1636803F00C03042B9DD0FFF7A2
:100AE400E1FBC01B4045F5D90320BDE8F081022A93
:100AF40002D113F0007FDFE713F0020FDCE7022BD3
:100B04000FD1636803F00C03082B86D0FFF7CAFBF0
:100B1400C01B4045F5D9E7E7FFF7C4FBC01B4045C0
:100B2400E2D8636813F00C0FF6D176E7136823F06C
:100B3400070333431360136803F007039E429CD1F9
:100B440072E76368E96823F4E0630B43636071E769
:100B54000020024000100240EB3100080C0000208D
:100B6400044B054A5B68C3F30223D35C034A106851
:100B7400D840704700100240FB3100080C000020F0
:100B8400044B054A5B68C3F3C223D35C034A106871
:100B9400D840704700100240FB3100080C000020D0
:100BA40003680020DA6842F00102DA601A6842F051
:100BB40001021A60704770477047704770470368B6
:100BC40010B51A69044691070ED5DA6892070BD559
:100BD4006FF002021A6101229B6902779B0777D0AA
:100BE400FFF7EAFF0023237723681A69500710D51B
:100BF400DA6851070DD56FF004021A6102229B696D
:100C0400227713F4407F204668D0FFF7D5FF0023F6
:100C1400237723681A6912070FD5DA6810070CD5F1
:100C24006FF008021A610422DB69227799072046D3
:100C34005AD0FFF7C1FF0023237723681A69D2062D
:100C440010D5DA68D0060DD56FF010021A610822AB
:100C5400DB69227713F4407F20464BD0FFF7ACFFCB
:100C64000023237723681A69D10708D5DA68D207E5
:100C740005D56FF0010220461A6100F0BFFC23681D
:100C84001A69100608D5DA68110605D56FF08002D6
:100C940020461A6100F0BFF823681A69520608D585
:100CA400DA68500605D56FF0400220461A61FFF756
:100CB40085FF23681A69910622D5DA6892061FD542
:100CC4006FF020022046BDE810401A6100F0A2B87F
:100CD400FFF771FF2046FFF770FF83E7FFF76BFF15
:100CE4002046FFF76AFF92E7FFF765FF2046FFF70C
:100CF40064FFA0E7FFF75FFF2046FFF75EFFAFE763
:100D040010BD0000244A0368904212D002F500622C
:100D140090420ED0B0F1804F0BD0A2F598329042A1
:100D240007D002F58062904203D002F580629042BF
:100D34001DD14A6823F070031343174A904212D01E
:100D440002F5006290420ED0B0F1804F0BD0A2F5B4
:100D54009832904207D002F58062904203D002F5A7
:100D64008062904203D1CA6823F4407313434A69F2
:100D740023F08003134303608B68C3620B688362B0
:100D8400054B984203D003F50063984201D10B69E7
:100D94000363012343617047002C014010B50446EE
:100DA400A0B190F83D3003F0FF021BB980F83C205D
:100DB40001F000F80223206884F83D30211DFFF77C
:100DC400A1FF0123002084F83D3010BD012010BD97
:100DD40090F83C3010B5012B4FF0020318D080F886
:100DE4003D3003680C685A68496822F070025A6002
:100DF4005A6822435A609A6822F080029A609A687C
:100E04000A439A60012380F83D30002380F83C3087
:100E1400184610BD704770470368DA6822F4907270
:100E2400DA605A6922F001025A61202380F83A30CC
:100E3400704700002DE9F0470568C2682B69016915
:100E440023F4405313432B618368EA680B434169DD
:100E540022F4B05222F00C020B431343EB606B6993
:100E6400826923F4407313436B61404B81469D4276
:100E74004FF0190446D1FFF783FE04FB00F3D9F8C1
:100E840004604FF06408B600B3FBF6F3B3FBF8F369
:100E94001E01FFF775FE6043D9F804309B00B0FBD8
:100EA400F3F7FFF76DFE6043D9F804309B00B0FB05
:100EB400F3F3B3FBF8F308FB13731B013233B3FBF7
:100EC400F8F303F0F007FFF75BFE6043D9F8042062
:100ED4009200B0FBF2FAFFF753FE6043D9F80430F6
:100EE4009B00B0FBF3F3B3FBF8F308FB13A31B0164
:100EF4003233B3FBF8F303F00F033B433344AB60EB
:100F0400BDE8F087FFF72CFE04FB00F3D9F804607A
:100F14004FF06408B600B3FBF6F3B3FBF8F31E011D
:100F2400FFF71EFE6043D9F804309B00B0FBF3F7D3
:100F3400FFF716FE6043D9F804309B00B0FBF3F3CF
:100F4400B3FBF8F308FB13731B013233B3FBF8F361
:100F540003F0F007FFF704FE6043D9F80420920081
:100F6400B0FBF2FAFFF7FCFDB7E700BF0038014021
:100F7400F8B504460E4617461D4621680B6836EA46
:100F8400030301D10020F8BD6B1CF7D095B9236889
:100F94000320DA6822F4D072DA605A6922F001027E
:100FA4005A61202384F8393084F83A30002384F8D5
:100FB4003830F8BDFFF776F9C01B8542DDD2E6E78D
:100FC40010B5044640B390F8393003F0FF021BB962
:100FD40080F8382000F002FF2423226884F8393096
:100FE400D368204623F40053D360FFF723FF23681C
:100FF40000201A6922F490421A615A6922F02A02E6
:101004005A61DA6842F40052DA602023E06384F81B
:10101400393084F83A3010BD012010BD2DE9F0417B
:101024001F4690F839300446202B0D4690464ED189
:10103400002949D0002A47D090F83830012B46D0F7
:10104400012380F838300023C363212380F839302A
:10105400FFF728F90646A4F82480A4F82680E38C38
:101064009BB26BB93B46324640212046FFF780FFD6
:10107400A8B9202384F8380084F83930BDE8F08119
:10108400E38C3246013B9BB2E384A3688021B3F531
:10109400805F20463B460ED1FFF76AFF10B1032064
:1010A400BDE8F0812B882268C3F3080353602369E9
:1010B40043B90235D3E7FFF75BFF0028EFD123687C
:1010C4002A785A600135CAE70120BDE8F081022080
:1010D400BDE8F08190F83A30202B20D1E9B1E2B19B
:1010E40090F83830012B1AD0C28582850023222241
:1010F400C36380F83A2002688162D16880F838308E
:1011040041F48071D1605169184641F00101516187
:10111400D16841F02001D16070470120704702205E
:101124007047704790F83A3010B5222B36D1836857
:101134000169B3F5805F0268836A23D15268E9B913
:10114400C2F3080223F8022B8362C48D013CA4B2CB
:10115400C4858CB90368DA6822F02002DA60DA68A0
:1011640022F48072DA605A6922F001025A61202363
:1011740080F83A3000F0C6F9002010BDD2B223F84E
:10118400012BE1E721B9591C526881621A70DCE72E
:101194005268591C816202F07F02F7E7022010BDF9
:1011A40070470000036870B51A6804461607D968CA
:1011B4005D6907D196065AD58D0658D5BDE87040AD
:1011C400FFF7B0BF15F0010502D111F4907F4ED0A6
:1011D400D30705D5CE0542BFE36B43F00103E363B8
:1011E400500704D51DB1E36B43F00203E363930797
:1011F40004D51DB1E36B43F00403E363160704D580
:101204001DB1E36B43F00803E363E36B002B66D08B
:10121400950604D5880602D52046FFF783FF236888
:1012240020465D69E26B110702D415F040051AD01F
:10123400FFF7F2FD23685A69520610D55A69606BAC
:1012440022F040025A6150B1254B4363FFF7AAF8DC
:10125400002844D0606BBDE87040436B18472046BB
:10126400FFF79EFF70BDFFF79BFFE56370BD160699
:1012740027D50D0625D594F83920212A2FD1A26827
:10128400B2F5805F226A17D11188C1F30801596051
:10129400216979B902322262E28C013A92B2E28483
:1012A400EAB9DA6822F08002DA60DA6842F04002D1
:1012B400DA6070BD0132EEE7511C216212785A6087
:1012C400EAE750060BD54A0609D5DA68204622F02B
:1012D4004002DA60202384F83930FFF722FF70BD22
:1012E400E912000808B50023406AC385C384FFF7E8
:1012F40057FF08BD4378013B052B10D8DFE803F006
:101304000603060F090B0A2100F08CB9072100F02F
:1013140091B90F21F8E781780331C9B2F4E7704736
:101324002DE9F8438179C379C278254D43EA012335
:1013340025F81230017A437AC278224C43EA012319
:1013440024F81230867AC37AC2781F4943EA062306
:1013540021F8123000221D4B1D4E18781D4FDFF866
:1013640080E0DFF880C0D3B2834207D300224FF479
:1013740080511948FFF770F901221AE0935D37F89C
:10138400139035F81380C1450CD23EF8139034F80D
:101394001380C14506D23CF8138031F81330013272
:1013A4009845E0D301224FF480510B48FFF754F9DC
:1013B4000022BDE8F8434FF400510848FFF74CB948
:1013C400F4000020E2000020D0000020C60000202D
:1013D400C7000020B4000020000C014000080140B8
:1013E400A20000209000002030B545789BB0044650
:1013F4006422002101A800F01EFE6B1E052B11D8EB
:10140400DFE803F0031521333A4CA178601C00F0A7
:1014140077FC6071A2882068A3790190ADF8082058
:101424008DF80A3001A8FFF765FF1BB030BDA27824
:101434002146033201A800F0F3FDE3792B4A8DF82D
:101444000B301370EEE7012000F0E6F8A278214695
:10145400033201A800F0E4FD9DF806100DF105002B
:1014640000F04EFC8DF80900DCE7214AE07813789F
:101474002049C8540133E4E7A2782146033201A885
:1014840000F0CEFD9DF806100DF1050000F038FCCB
:101494008DF809002046FFF743FFC3E7A2782146F1
:1014A400033201A800F0BCFD22796379A17A43EAF2
:1014B4000223114A0DF1050022F81130A279E379D3
:1014C400A17A43EA02230D4A22F81130227A637A80
:1014D400A17A43EA02230A4A22F811309DF8061041
:1014E40000F00EFC8DF80F009CE700BF0C010020FB
:1014F400C6000020C7000020B4000020A200002085
:101504009000002002682E4B10B59A4204461AD16E
:101514002C4A2D49137808782C49EB28C85403F138
:101524000103DBB2137009D18978033B99420BBFE5
:1015340001220023264B137008BF1A70012222498E
:101544002448FFF7C7FD2268234B9A4217D123484A
:10155400234B01781A781D4BEB2A5A5401F10101EF
:10156400C9B2017006D19A78CB1E9A4222D10222C6
:10157400174B1A7001221A491A48FFF7ABFD22686B
:10158400194B9A421BD1194A194912780B780F4802
:10159400EB2AC25408BF032203F101030B7008BFF6
:1015A4000B4B124908BF1A7012480122BDE81040C3
:1015B400FFF790BD0439104800F046FDDAE710BD8E
:1015C4000038014072010020740200200E01002046
:1015D40088010020D0010020004400407301002055
:1015E400CD010020B802002000480040CC010020BA
:1015F400740100208C0100202C3100080268044B87
:101604009A4201BF034A136801331360704700BF55
:101614000010004008010020014B1870704700BF03
:101624000D0100200A460A2301460148FFF7F6BCD3
:101634008C0100200A460A2301460148FFF7EEBC4C
:10164400D001002010B514460A230248FFF7E6FC37
:10165400204610BD8C010020F8B5174C0646A17831
:10166400601C63185A7800F066FB2546D0B9134F06
:101674003378441CC0B283420ED8AB7800211D4499
:101684006A780F4800F0E0FC0021642231700A48B7
:10169400BDE8F84000F0CFBC295C384600F0D4FC2B
:1016A4002046E5E7012803D12046FFF79DFEEBE73E
:1016B400044800F03DFDE7E70E0100203631000844
:1016C4003C3100086231000808B5082800F2228184
:1016D400DFE810F00900390063006D007D0093001D
:1016E400AD00CD00F30001224FF400518A48FEF70B
:1016F400B3FF01224FF480418748FEF7ADFF01227A
:101704004FF400418448FEF7A7FF0122402183489B
:10171400FEF7A2FF012280218048FEF79DFF0122EF
:101724004FF480717D48FEF797FF01224FF400715A
:101734007A48FEF791FF01224FF480717848BDE8A2
:101744000840FEF789BF01224FF400517248FEF7AA
:1017540083FF00224FF480416F48FEF77DFF002293
:101764004FF400416C48FEF777FF002240216B489C
:10177400FEF772FF002280216848FEF76DFF002209
:101784004FF480716548FEF767FF00224FF4007143
:101794006248FEF761FF0022CEE701224FF4804148
:1017A4005D48FEF759FF01224FF40051D4E70122AE
:1017B4004FF400415848FEF74FFF01224FF4804197
:1017C4005548FEF749FF01224FF40051CAE70122B0
:1017D40040215248FEF740FF01224FF480414E4819
:1017E400FEF73AFF01224FF400514B48FEF734FF55
:1017F40001224FF400414848BAE7012280214748BA
:10180400FEF72AFF01224FF480414348FEF724FFEC
:1018140001224FF400514048FEF71EFF01224FF40D
:1018240000413D48FEF718FF01224021A4E70122B0
:101834004FF480713948FEF70FFF01224FF48041C5
:101844003548FEF709FF01224FF400513248FEF7F4
:1018540003FF01224FF400412F48FEF7FDFE012251
:1018640040212E48FEF7F8FE012280218AE701225A
:101874004FF400712948FEF7EFFE01224FF4804136
:101884002548FEF7E9FE01224FF400512248FEF7F5
:10189400E3FE01224FF400411F48FEF7DDFE012262
:1018A40040211E48FEF7D8FE012280211B48FEF786
:1018B400D3FE01224FF480716AE701224FF4807154
:1018C4001748FEF7C9FE01224FF480411248FEF783
:1018D400C3FE01224FF400510F48FEF7BDFE012262
:1018E4004FF400410C48FEF7B7FE012240210B489B
:1018F400FEF7B2FE012280210848FEF7ADFE012268
:101904004FF400710548FEF7A7FE01224FF48071E1
:10191400024814E708BD00BF000C0140001001405C
:101924000008014010B590B02822002106A800F05C
:1019340082FB0021142201A800F07DFB0224012275
:101944004FF4803306A8069207930A920E930D94DF
:10195400FEF78CFE0F23002101934FF4806301A84E
:101964000294039104930591FFF748F810B010BD59
:101974002DE9F04F04244FF00108BE27B84EDFF8DC
:101984004CA333788FB08DF81B309AF80030214681
:101994000DF119008DF818708DF819808DF81A4022
:1019A4008DF81C3000F0ACF90323EB258DF82130C1
:1019B400337821468DF823309AF800308DF81D00D5
:1019C4000DF121008DF824308DF81E508DF8207013
:1019D4008DF8224000F094F98DF826508DF82500FA
:1019E400FEF742FCFFF79EFF102200210AA800F038
:1019F40022FB9C4B4BF6D8719A699B4842F010022B
:101A04009A619A69022502F010020292029A9A6976
:101A1400DFF8BC9242F020029A619A69934F02F077
:101A240020020392039A9A694FF00C0B22439A61A5
:101A34009A698F4E22400492049A9A69002442F0D3
:101A440008029A619B69002203F008030593059B31
:101A5400FEF702FE002242F2F0118648FEF7FCFD7A
:101A640000224FF470418448FEF7F6FD4BF6D8731C
:101A74000AA97D480A93CDF82C800D950C94FEF7A5
:101A8400FFFC42F2F0130AA97A480A93CDF82C809D
:101A94000D950C94FEF7F4FC4FF470430AA97648B4
:101AA4000A93CDF82C800D950C94FEF7E9FC40F2D6
:101AB4003F63724A484689E80C000923C9F8084084
:101AC400C9F80C30C9F818400A940B94FFF766F96A
:101AD4000AA948460A940B94FFF77AF9684B3846EA
:101AE4003B604FF4E133BC607B600193FC603C617C
:101AF400C7F814B0BC61FC61FFF762FA614A019B4C
:101B0400614D304632607360B460F4603461C6F88D
:101B140014B0B461F461FFF753FA019B5B4A2846A1
:101B24006B602A60AC60EC602C61C5F814B0AC61E9
:101B3400EC61FFF745FA224621462720FEF7DCFB3D
:101B44002720FEF70DFC224621462520FEF7D4FB74
:101B54002520FEF705FC224621462620FEF7CCFB75
:101B64002620FEF7FDFB224621463620FEF7C4FB65
:101B74003620FEF7F5FB4846FFF712F84246444983
:101B84003846FFF7A7FA424642493046FFF7A2FA21
:101B9400424641492846FFF79DFA404B21461B68BF
:101BA4003F4E986800F0CCFA3E4800F0C1FA3E4837
:101BB40000F0BEFA3D4A3E493E4800F045FA3E4830
:101BC40000F0B6FA374800F0B3FA86F80080DFF880
:101BD40004815546C246DFF8909098F8003083B1EE
:101BE400012B06D13548FFF737FD00238AF8003072
:101BF400F3E7022B01D13248F5E7032BF5D1314845
:101C0400F1E7314F3A68B2F5FA7FE6D996F800B0B9
:101C1400BBF1010F60D1287808280DD9184633701C
:101C2400FFF752FD85F800B04FF400414846FEF737
:101C340018FD00233B60D0E7FFF746FD4FF4FA7030
:101C4400FEF736FB08A8FFF7CFFB4FF4FA70FEF758
:101C54002FFB2B785A1C2A708DF82430E4E700BF40
:101C64000C0100200010024000100140D0010020AF
:101C7400B802002000080140000C014000100040A0
:101C840000380140004400408C010020004800401E
:101C940074020020CD010020CC010020100000209F
:101CA4000D010020703100089A310008A7310008A6
:101CB400B0310008BC310008CD31000872010020A9
:101CC4007301002074010020080100200800002096
:101CD400780200208801002006A8FFF785FB064A49
:101CE400631C125DDBB28DF81C20044A14789C42FC
:101CF400CCBF1C46002497E7C7000020C600002084
:101D040010B5FF230446221AD2B2914201D81846D4
:101D140010BD14F8012B5340082213F0800F02F178
:101D2400FF324FEA430318BF83F0310312F0FF027E
:101D3400DBB2F2D1E7E730B5FF2305462C1AE4B253
:101D4400A14203D89B1A5842584130BD15F8014BA3
:101D54006340082413F0800F04F1FF344FEA430377
:101D640018BF83F0310314F0FF04DBB2F2D1E5E7CE
:101D74000E4B82B09A6942F001029A619A6902F0AC
:101D840001020092009ADA6942F08052DA61DB695A
:101D9400074A03F080530193019B536823F0E063E7
:101DA40043F08063536002B0704700BF00100240EC
:101DB400000001400268084B82B09A420AD103F540
:101DC4000033DA6942F01002DA61DB6903F01003D0
:101DD4000193019B02B070470010004010B5044607
:101DE4008AB01022002106A800F025F923683D4A94
:101DF40093422AD13C4B06A99A693C4842F480425A
:101E04009A619A6902F480420092009A9A6942F0B7
:101E140004029A619B6903F004030193019B4FF44C
:101E2400007306930223079303230993FEF728FB09
:101E34004FF4806306930023079301232B480893F0
:101E440006A9FEF71DFB0AB010BD294A93421ED114
:101E5400254B06A9DA69254842F40032DA61DA69C9
:101E640002F400320292029A9A6942F004029A61E0
:101E74009B6903F004030393039B04230693022347
:101E8400079303230993FEF7FBFA0823D2E7194AC1
:101E94009342D8D1144B06A9DA69174842F4802238
:101EA400DA61DA6902F480220492049A9A6942F0AF
:101EB40008029A619B6903F008030593059B4FF49C
:101EC400806306930223079303230993FEF7D8FA4A
:101ED4004FF40063069300230793012306A9089394
:101EE4000548AEE7003801400010024000080140F8
:101EF4000044004000480040000C01407047FEE7E9
:101F0400FEE7FEE7FEE7704770477047FEF7BEB98D
:101F14000148FFF747B900BFD00100200148FFF78F
:101F240041B900BFB80200200148FFF73BB900BF28
:101F34008C0100200148FEF742BE00BF7802002059
:101F44000F4B1A6842F001021A6059680D4A0A40A0
:101F54005A601A6822F0847222F480321A601A6875
:101F640022F480221A605A6822F4FE025A604FF466
:101F74001F029A604FF00062034B9A60704700BFE3
:101F8400001002400000FFF800ED00E0002103E033
:101F94000B4B5B58435004310A480B4B42189A428E
:101FA400F6D30A4A02E0002342F8043B084B9A4263
:101FB400F9D3FFF7C5FF00F00FF8FFF7D9FC70471E
:101FC400A4320008000000207400002074000020E7
:101FD400FC020020FEE7000070B500250C4E0D4CFD
:101FE400A41BA410A54209D101F08AF800250A4EC9
:101FF4000A4CA41BA410A54205D170BD56F8253087
:1020040098470135EEE756F8253098470135F2E751
:102014009C3200089C3200089C320008A032000860
:1020240010B5431E0A44914200D110BD11F8014B72
:1020340003F8014FF7E703460244934200D1704787
:1020440003F8011BF9E700000FB40A4B13B51C6831
:1020540024B1A36913B9204600F0DAFA05AB049A57
:10206400A1682046019300F09BFC02B0BDE810403B
:1020740004B070471000002070B50E46054618B134
:1020840083690BB900F0C4FAAB69AC6813B928468C
:1020940000F0BEFA234B9C4217D16C68A3891B073E
:1020A4001DD52369DBB1013EA36816F8011F013B6E
:1020B400A360E9B9002B2EDA22460A21284600F053
:1020C400F5F8013011D00A2070BD174B9C4201D1A4
:1020D400AC68E3E7154B9C4208BFEC68DEE7214699
:1020E400284600F035F90028DDD04FF0FF3070BDF0
:1020F400002B04DAA269934206DB0A2904D0236880
:102104005A1C22601970CFE72246284600F0CEF808
:102114000130C9D1E9E70A2023685A1C22601870EB
:1021240070BD00BF28320008483200080832000899
:10213400024B01461868FFF79FBF00BF1000002044
:1021440000294FF480630CBF0222002200F000B883
:102154002DE9F7431D46514B04461E680F46904631
:1021640026B1B36913B9304600F052FA4C4B9C4285
:1021740052D17468B8F1020F06D0B8F1010F00F221
:102184008980002DC0F286802146304600F0D6F9C1
:10219400616B41B104F14403994202D0304600F02E
:1021A4002DFB002363630023A3616360A3891B06E3
:1021B40003D52169304600F021FBA389B8F1020F51
:1021C40023F44A6323F00303A3815DD001AB6A4681
:1021D4002146304600F0A6FAA3891843A0812DBBFE
:1021E400009D284600F002FB074600284ED1DDF88A
:1021F4000090A9453CD14FF0FF30A38943F002037E
:10220400A3810023A36004F1470323602361012316
:10221400636103B0BDE8F083224B9C4201D1B468F2
:10222400A8E7214B9C4208BFF468A3E7002FD8D04D
:10223400B36913B9304600F0EBF9B8F1010F08BFE8
:10224400A389276004BF43F00103A381A389276105
:1022540013F0080065611BD013F001004FF0000378
:102264001FBF6D42A360A561184608BFA560D0E7F3
:10227400484600F0BBFA07460028BCD0A3894D4667
:1022840043F08003A381D3E70020B6E7A946F5E72E
:10229400A060BEE74FF0FF30BBE700BF1000002096
:1022A400283200084832000808320008F8B50E4603
:1022B4001446054618B183690BB900F0A9F9214BFE
:1022C4009C422AD16C68A369A360A3891A072ED5FE
:1022D400236963B323692068F6B2C01A6369374679
:1022E400984204DB2146284600F028F928BBA3685D
:1022F4000130013BA36023685A1C22601E7063698D
:10230400984204D0A389DB0719D50A2E17D1214698
:10231400284600F013F990B10FE00B4B9C4201D119
:10232400AC68D0E7094B9C4208BFEC68CBE7214678
:10233400284600F00DF80028CCD04FF0FF3738467F
:10234400F8BD00BF283200084832000808320008EF
:10235400324B70B51D6806460C4625B1AB6913B9FE
:10236400284600F055F92E4B9C420FD16C68B4F905
:102374000C309AB215072CD4D00611D4092232603D
:1023840043F04003A3814FF0FF3070BD254B9C42C6
:1023940001D1AC68EBE7244B9C4208BFEC68E6E74C
:1023A400510712D5616B41B104F14403994202D043
:1023B400304600F023FA00236363A38923F0240347
:1023C400A3810023636023692360A38943F0080386
:1023D400A38123694BB9A38903F42073B3F5007F68
:1023E40003D02146304600F0C1F9A28912F001035E
:1023F4000CD00023A36063695B42A361236953B9D2
:10240400B4F90C3013F08000BAD170BD920758BFF4
:102414006369A360F2E70020F7E700BF1000002023
:102424002832000848320008083200088A892DE959
:10243400F041054610070C465AD44B68002B05DCC6
:102444000B6C002B02DC0020BDE8F081E66A002E54
:10245400F9D0002312F480522F682B6033D0606DC2
:10246400A3895A0705D56368C01A636B0BB1236C43
:10247400C01A00230246E66A216A2846B047431C74
:10248400A38906D129681D294BD82B4ACA40D607EF
:1024940047D5002262602269D904226004D5421C17
:1024A40001D12B6803B96065616B2F600029CAD024
:1024B40004F14403994202D0284600F09FF9002019
:1024C4006063BDE8F081216A01232846B047411CBE
:1024D400C6D12B68002BC3D01D2B01D0162B01D1E4
:1024E4002F60B0E7A38943F04003A381BDE8F081E6
:1024F4000F69002FA7D0930718BF00230E6808BFE9
:102504004B69A6EB07080F608B60B8F1000F9ADDEA
:1025140043463A46216A2846A66AB047002807DCA3
:10252400A38943F04003A3814FF0FF30BDE8F0815D
:102534000744A8EB0008E8E70100402038B50B6920
:1025440005460C46DBB118B183690BB900F060F89D
:102554000C4B9C4209D16C68B4F90C307BB1214618
:102564002846BDE83840FFF761BF074B9C4201D1C4
:10257400AC68F1E7054B9C4208BFEC68ECE700202F
:1025840038BD00BF2832000848320008083200086D
:10259400014900F0A9B800BF41250008002310B587
:1025A400044603604360836081814366C2810361A2
:1025B40043618361194608225C30FFF73CFD054BFB
:1025C40024626362044BA362044BE362044B2363FF
:1025D40010BD00BF212F0008432F00087B2F0008E7
:1025E4009F2F000870B568254A1E55430E4605F115
:1025F400740100F04FF9044640B1002180E8420024
:102604000C30A06005F16802FFF715FD204670BD8F
:10261400836910B5044633BB8364C3640365124BFA
:10262400124A1B688262984204BF0123836100F04E
:102634001FF86060204600F01BF8A060204600F000
:1026440017F80022E06004216068FFF7A7FF012269
:102654000921A068FFF7A2FF02221221E068FFF718
:102664009DFF0123A36110BD0432000895250008D5
:10267400F8B51C4B07461E68B36913B93046FFF71B
:10268400C7FF4836B4687368013B03D5336833B178
:102694003668F7E7B4F90C506DB16834F4E70421F7
:1026A4003846FFF79FFF30600028F1D10C23044621
:1026B4003B602046F8BD4FF6FF73E3810123656656
:1026C400A3812560A560656025616561A561082217
:1026D400294604F15C00FFF7AEFC6563A563A564BD
:1026E400E564E6E7043200082DE9F84380468946AC
:1026F400002600F1480414B93046BDE8F883A56803
:102704006768013F01D52468F5E7AB89012B07D938
:10271400B5F90E30013303D029464046C847064375
:102724006835EEE770B50E46B1F90E1090B0002989
:1027340014461D4607DA00232B60B3891A0610D409
:102744004FF480630EE001AA00F04EFC0028F2DB97
:10275400029A02F47042A2F500535A425A412A6086
:10276400EEE740230020236010B070BD8B8973B561
:102774009D0706460C4607D504F1470323602361F1
:102784000123636102B070BD01AB6A46FFF7CAFF63
:1027940000990546304600F07DF848B9B4F90C308C
:1027A4009A05EFD423F0030343F00203A381E3E784
:1027B4000D4BB362A389206043F08003A381009B87
:1027C40020616361019B5BB1B4F90E10304600F0E7
:1027D4001DFC28B1A38923F0030343F00103A38163
:1027E400A3891D43A581CDE795250008024B014629
:1027F400186800F04FB800BF1000002038B5054637
:10280400002943D051F8043C0C1F002BB8BFE41836
:1028140000F02CFC1E4A1368104633B96360146040
:102824002846BDE8384000F022BCA3420BD92168F9
:102834006218934201BF1A685B6852182260636091
:102844000460EDE713465A680AB1A242FAD919683E
:102854005818A0420BD120680144581882421960CC
:10286400DED110685268014419605A60D8E702D971
:102874000C232B60D4E7206821188A4201BF116819
:1028840052680918216062605C60C9E738BD00BF06
:102894007801002070B5CD1C25F0030508350C2DFA
:1028A40038BF0C25002D064601DBA94203D90C23B1
:1028B4003360002070BD00F0D9FB234A1468214620
:1028C40091B9224C23681BB9304600F017FB2060F5
:1028D4002946304600F012FB431C26D10C23304617
:1028E400336000F0C4FBE4E70B685B1B1AD40B2BCA
:1028F4000FD90B60CC18CD50304600F0B8FB04F172
:102904000B00231D20F00700C31A1BD05A42E250CB
:1029140070BD8C420BBF63684B681360636018BF63
:102924000C46E9E70C464968CAE7C41C24F00304D2
:10293400A04205D0211A304600F0E0FA0130CDD093
:102944002560D9E770BD00BF780100207C0100201C
:10295400936810B4013B002B936008DA9469A34296
:1029640002DBCBB20A2B02D110BCFFF79FBC136869
:10297400581C10601970C8B210BC7047F8B50646F0
:102984000F461446D518AC4201D1002007E03A4660
:1029940014F8011B3046FFF7DBFF431CF3D1F8BDED
:1029A4002DE9F04F9DB00C4617460393064618B127
:1029B40083690BB9FFF72CFE7C4B9C4257D174689A
:1029C400A38918075DD52369002B5AD000230993E6
:1029D40020238DF8293030234FF0010B8DF82A3055
:1029E400B846454615F8013B002B55D1B8EB070A0C
:1029F4000BD053463A4621463046FFF7BFFF01301D
:102A040000F0C480099B5344099398F80030002BCC
:102A140000F0BC8000234FF0FF320493079305922B
:102A240006938DF853301A9305222978604800F0F4
:102A34000FFB05F10108049B002831D1D90644BFDE
:102A440020228DF853201A0744BF2B228DF85320DF
:102A54002A782A2A2CD000210A20079AA84698F816
:102A640000300135303B092B6DD971B326E0514B51
:102A74009C4201D1B468A3E74F4B9C4208BFF46861
:102A84009EE721463046FFF763FC00289ED04FF0B6
:102A9400FF301DB0BDE8F08F252BA7D0A846A0E7D6
:102AA400434A4546801A0BFA00F018430490BBE7EA
:102AB400039A111D12680391002A01DB079204E0B6
:102AC400524243F002030792049398F800302E2BED
:102AD40010D198F8013008F101012A2B37D1039B5A
:102AE40008F102081A1D1B680392002BB8BF4FF0AF
:102AF400FF330593314D032298F80010284600F067
:102B0400A7FA40B14023401B03FA00F0049B08F1EC
:102B140001080343049398F800100622284808F19A
:102B240001078DF8281000F093FA002834D0254BC3
:102B340003BB039B073323F0070308330393099B69
:102B44004B4409934CE700FB0232012186E7002342
:102B54000A2518460593884698F800200131303A32
:102B6400092A03D9002BC5D00590C3E705FB002033
:102B74000123F0E703AB00932246134B04A930462C
:102B8400AFF30080B0F1FF3F8146D8D1A3895B0643
:102B94003FF57DAF09987CE703AB009322460A4BCF
:102BA40004A9304600F08AF8ECE700BF2832000898
:102BB4006832000848320008083200086E32000803
:102BC4007232000800000000812900082DE9F04756
:102BD40091461F468A680B6906469342B8BF13465E
:102BE400C9F8003091F843200C46DDF8208012B17A
:102BF4000133C9F800302368990642BFD9F8003080
:102C04000233C9F80030256815F0060507D104F130
:102C1400190AE368D9F800209B1A9D422ADB94F82C
:102C240043302268003318BF012392062FD404F1E5
:102C3400430239463046C047013022D02368E56854
:102C440003F00603042B18BF0025D9F800204FF029
:102C5400000908BFAD1AA368226908BF25EAE57513
:102C64009342C4BF9B1AED181A344D451BD1002062
:102C7400BDE8F0870123524639463046C04701304B
:102C840003D14FF0FF30BDE8F0870135C1E73020B4
:102C9400E11881F843005A1C94F845102244023389
:102CA40082F84310C3E70123224639463046C04721
:102CB4000130E6D009F10109D7E700002DE9F0431E
:102CC40017460A7E85B06E2A984606460C460C9B2B
:102CD40001F1430E00F0BC801AD8632A2ED00AD822
:102CE400002A00F0C880582A00F08A8004F14205C6
:102CF40084F842202AE0642A01D0692AF6D12168A6
:102D04001A6811F0800F23D0111D1960136827E091
:102D1400732A00F0B48008D86F2A2AD0702AE5D12B
:102D24000A6842F020020A6003E0752A21D0782A5A
:102D3400DCD178226F4984F8452064E01A6801F1F7
:102D44004205111D1960136884F842300123A3E081
:102D540011F0400F02F104011960D7D0B2F900302C
:102D6400002B03DA2D225B4284F8432062490A22B5
:102D740017E02068196810F0800F03D0081D186050
:102D84000B6806E010F0400F01F104001860F7D062
:102D94000B886F2A14BF0A2208225749002084F89E
:102DA40043006568002DA560C0F29C80206820F077
:102DB40004002060002B3FD1002D40F09580754623
:102DC400082A0BD12368DA0708D5236962689A4276
:102DD400DEBF302305F8013C05F1FF35AEEB0503FA
:102DE4002361CDF800803B4603AA21463046FFF715
:102DF400EDFE013055D14FF0FF3005B0BDE8F08352
:102E040081F845203C492268186812F0800F00F1CF
:102E140004051D6001D0036802E05506FBD5038854
:102E2400D00744BF42F0200222601BB9226822F07E
:102E3400200222601022B1E77546B3FBF2F002FBD8
:102E44001033CB5C05F8013D03460028F5D1B7E704
:102E540008681A6810F0800F496904D0101D1860C2
:102E64001368196007E010F0400F02F104001860C5
:102E74001368F6D01980002375462361B1E71A68F8
:102E8400111D1960156800216268284600F0E0F8F9
:102E940008B1401B606063682361002384F84330F9
:102EA4009FE723692A4639463046C0470130A2D0FD
:102EB40023689B0707D5002504F11909E368039AE1
:102EC4009B1A9D4205DBE068039B9842B8BF1846F5
:102ED40093E701234A4639463046C04701308AD039
:102EE4000135EBE7002BA7D10B7804F1420584F8F8
:102EF400423065E78A3200087932000838B5002389
:102F0400054C05460846236000F0ECF8431C02D14A
:102F1400236803B12B6038BDF802002010B50C46BD
:102F2400B1F90E1000F0A4F80028ABBF636DA389BB
:102F34001B1823F48053ACBF6365A38110BD2DE936
:102F4400F0411F468B890546DB050C46164605D520
:102F540002230022B1F90E1000F068F8A38932466A
:102F640023F48053A381B4F90E103B462846BDE8F0
:102F7400F04100F017B810B50C46B1F90E1000F08E
:102F840055F8431CA38915BF606523F4805343F4AB
:102F94008053A38118BFA38110BDB1F90E1000F0B6
:102FA40013B8000038B50546084611460022054C02
:102FB40022601A46FEF746FB431C02D1236803B184
:102FC4002B6038BDF802002038B50023054C0546B7
:102FD4000846236000F05EF8431C02D1236803B165
:102FE4002B6038BDF802002038B50023064C054696
:102FF40008461146236000F055F8431C02D12368AB
:1030040003B12B6038BD00BFF802002038B500239F
:10301400054C05460846236000F04CF8431C02D1D9
:10302400236803B12B6038BDF802002038B505468B
:10303400084611460022054C22601A4600F042F868
:10304400431C02D1236803B12B6038BDF802002071
:1030540010B5C9B202449042034601D1002010BD0C
:103064001C7801308C42F6D1184610BD7047704769
:1030740038B50546084611460022054C22601A461A
:1030840000F028F8431C02D1236803B12B6038BD3B
:10309400F80200205822024B4FF0FF301A607047AC
:1030A400F80200205822024B4FF0FF301A6070479C
:1030B400F80200205822024B00201A60704700BF1B
:1030C400F80200205822024B4FF0FF301A6070477C
:1030D400F80200205822024B4FF0FF301A6070476C
:1030E400F8020020044B0246196809B90349196023
:1030F400186802441A60704780010020FC02002016
:10310400F8B500BFF8BC08BC9E467047F8B500BFD0
:08311400F8BC08BC9E467047A0
:10311C0002030405060708090A0B0C0D0E0F10100C
:10312C00554152542032202564002530327820003D
:10313C004F726967696E616C20435243203A2025B7
:10314C003032782052656376435243203A20253042
:10315C003278200D0A0057686174204861707065E0
:10316C006E3F0D002A2A2A2A2A2A2A2A2A2A2A2AA1
:10317C002A2A2A2A2A2A2A2A2A2A2A2A2A2A2A2AA3
:10318C002A2A2A2A2A2A2A2A2A2A2A2A0D00524795
:10319C00422050726F6A6563740D0031373A3437D0
:1031AC003A3136004D6172203138203230313900DD
:1031BC004275696C642061742025732025730D0A97
:1031CC0000436F7079726967687420286329203214
:1031DC003031392E20424C554543454C4C0D0000A6
:1031EC0000000000000000010203040607080900AB
:1031FC000000000102030400140000200000000085
:10320C0000000000000000000000000000000000B2
:10321C0000000000000000000000000000000000A2
:10322C000000000000000000000000000000000092
:10323C000000000000000000000000000000000082
:10324C000000000000000000000000000000000072
:10325C00000000000000000000000000232D302BB7
:10326C002000686C4C00656667454647003031327B
:10327C0033343536373839414243444546003031D2
:10328C003233343536373839616263646566000031
:04329C00090200081B
:0432A000E50100083C
:1032A40001000000100000000100000000A24A0418
:1032B40014000020000000002832000848320008F2
:1032C40008320008000000000000000000000000B8
:1032D40000000000000000000000000000000000EA
:1032E40000000000000000000000000000000000DA
:1032F40000000000000000000000000000000000CA
:1033040000000000000000000000000000000000B9
:0433140000000000B5
:0400000508001F913F
:00000001FF
